:02000000D52BFE
:10000800FF00030E8301D9000A08DA008A010B11E8
:10001800D60A0319D70A0B1C1628861A1528013088
:10002800D5000B105A088A00590E8300FF0E7F0E68
:020038000900BD
:04003A0000000800BA
:10003E00083083120313FC002330FD00FD0B25282E
:06004E00FC0B2528080050
:10005400103083120313FD00FD0B2E28000008004E
:100064007408F8027508031C750FF9027608031C5E
:10007400760FFA027708031C770FFB02F30D0730A3
:10008400FC00730DF80DF90DFA0DFB0D7408731CCB
:100094005928F8027508031C750FF9027608031C29
:1000A400760FFA027708031C770FFB026628F8071D
:1000B40075080318750FF90776080318760FFA0701
:1000C40077080318770FFB07F30DFC0B4328720D19
:1000D400F80DF90DFA0DFB0D7408731C7F28F80256
:1000E4007508031C750FF9027608031C760FFA02D3
:1000F4007708031C770FFB028C28F8077508031890
:10010400750FF90776080318760FFA0777080318AE
:10011400770FFB07F20D0730FC00720DF80DF90D97
:10012400FA0DFB0D7408721CA528F8027508031C4F
:10013400750FF9027608031C760FFA027708031C80
:10014400770FFB02B228F80775080318750FF90733
:1001540076080318760FFA0777080318770FFB075A
:10016400F20DFC0B8F28710DF80DF90DFA0DFB0D36
:100174007408721CCB28F8027508031C750FF90269
:100184007608031C760FFA027708031C770FFB022C
:10019400D828F80775080318750FF90776080318A7
:1001A400760FFA0777080318770FFB07F10D07306E
:1001B400FC00710DF80DF90DFA0DFB0D7408711C9E
:1001C400F128F8027508031C750FF9027608031C60
:1001D400760FFA027708031C770FFB02FE28F80754
:1001E40075080318750FF90776080318760FFA07D0
:1001F40077080318770FFB07F10DFC0BDB28700D54
:10020400F80DF90DFA0DFB0D7408711C1729F8028D
:100214007508031C750FF9027608031C760FFA02A1
:100224007708031C770FFB022429F80775080318C5
:10023400750FF90776080318760FFA07770803187D
:10024400770FFB07F00D0730FC00700DF80DF90D6A
:10025400FA0DFB0D7408701C3D29F8027508031C87
:10026400750FF9027608031C760FFA027708031C4F
:10027400770FFB024A29F80775080318750FF90769
:1002840076080318760FFA0777080318770FFB0729
:10029400F00DFC0B272970185D297408F807750800
:1002A4000318750FF90776080318760FFA0777080D
:0802B4000318770FFB07080097
:1002BC0083120313EE1B64290513652905176E1BA6
:1002CC00692985136A298517EE1A6E2905106F297D
:1002DC0005146E1A732985107429851458187829F9
:1002EC0085157929851105151D200511EE19802913
:1002FC000513812905176E198529851386298517FC
:10030C00EE188A2905108B2905146E188F29851073
:10031C00902985145818942985159529851105154A
:10032C001D200511581C9C291F209D292A200800DE
:10033C00FB09FA09F909F809F80A0319F90A03196A
:08034C00FA0A0319FB0A08007C
:100354008312031358106B08EE005E215814080032
:0E0364008312031354088A0053088200080015
:10037200831203137408003A031DD4297508003A46
:10038200031DD4297608003A031DD4297708003AC0
:10039200031DD429FF30F000FF30F100FF30F200DE
:1003A2007F30F3006D2A83120313FC01F71BFC0A52
:1003B200FD01FB01FA01F901F801730872047104ED
:1003C20070040319682A73087706A000A01BFD09B0
:1003D200F71FF629F409F509F609F709F40A0319D2
:1003E200F50A0319F60A0319F70AF31F032AF0099B
:1003F200F109F209F309F00A0319F10A0319F20AE1
:100402000319F30A73087704A000A01B242A3220E0
:10041200FC1B412AFD1F682AF009F109F209F309C0
:10042200F00A0319F10A0319F20A0319F30AF80987
:10043200F909FA09FB09F80A0319F90A0319FA0A70
:100442000319FB0A682AF71F3B2AF31B352A730894
:10045200FB007208FA007108F9007008F800F30155
:10046200F201F101F0010B2AF301F201F101F001B5
:10047200F00A0034F309F209F109F009FC17082A1D
:10048200F80A0319F90A0319FA0A0319FB0A74088C
:100492007802031D0B2A75087902031D0B2A7608C0
:1004A2007A02031D0B2A77087B02031D0B2AFB012C
:1004B200FA01F901F801F00A0319F10A0319F20A23
:1004C2000319F30AF31F0B2AA0012016FF34A0011F
:0A04D2007C1C6C2A9E21003E0800ED
:1004DC00802A803083120313EB00932AC030EB0088
:1004EC00932A9430EB00932AD430EB00932A80307B
:1004FC00EB00932A831203136B08013A03196F2A3A
:10050C006B08023A0319742A6B08033A0319772A09
:10051C006B08043A03197A2A7D2A6C03F0006B08E5
:10052C00F0077008EB0058147008EE005E215810AC
:0A053C006D08EE005E21581408005F
:1005460083120313E8016808A03EEA000A30F400AB
:10055600F501F601F7016308F0006408F10065088B
:10056600F2006608F300B9217808F0007908F10076
:100576007A08F2007B08F3003030F0076A0884003E
:10058600700880000A30F400F501F601F7016308EF
:10059600F0006408F1006508F2006608F300B9216E
:1005A6007008E3007108E4007208E5007308E600CD
:1005B600E80A8030F400803073067402031DED2AC9
:1005C6007208003C031DED2A7108003C031DED2A4C
:1005D6007008003C0318F42A093068020318F42A4C
:1005E600A62A0B30E900E7010930670203183A2B07
:1005F6006908043A0319042B6908083A0319042BFD
:100606001A2B680867020318112B0130EB00023021
:100616006907EC002C30ED006E22192B0130EB003F
:1006260002306907EC002030ED006E22E90368080D
:100636006702031C232B6708003A0319232B2F2B71
:100646000130EB0002306907EC006708A03E840029
:100656000008ED006E22372B0130EB0002306907EF
:10066600EC002030ED006E22E903E70AF72A0800C5
:100676004D2B803083120313E300602BC030E30060
:10068600602B9430E300602BD430E300602B803085
:10069600E300602B831203136308013A03193C2B12
:1006A6006308023A0319412B6308033A0319442BE2
:1006B6006308043A0319472B4A2B6403F0006308C6
:1006C600F0077008E3007008EE005E215810E6019E
:1006D60066086507840000080319792B6608650714
:1006E60084000008EB00AA21E60A6B2B58140800C8
:1006F600B2218A110A128000840AD30A0319D40A85
:08070600F003031D7B2B08002A
:10070E008316031305118511851005108513051326
:10071E0083120511851105138513051085101F20F1
:10072E001F201F200514851405151D2005111F20DF
:10073E0005151D2005111F2005151D2005111F2053
:10074E00851005151D2005111F2005151D200511ED
:10075E000510051705151D2005111F2005138514FD
:10076E0005151D200511851005151D2005111F20CD
:10077E0005151D200511851405151D2005111F20B9
:10078E00851005151D2005110517851705148514EF
:0C079E0005151D2005111F20581408002F
:1007AA003C250730831203139F000B30FB002630D1
:1007BA00FC005D30FD00FD0BE02BFC0BE02BFB0B7E
:1007CA00E02B000000000E309000303083168500C8
:1007DA00EF3086008312061687230130EE005E2171
:1007EA000C30EE005E210130E3000130E4003130CC
:1007FA00E5003B230230E3000130E4004530E50028
:10080A003B230630FB001330FC00AD30FD00FD0B2E
:10081A000C2CFC0B0C2CFB0B0C2C000000000130E8
:10082A00EE005E21E1010330610203182E2C18301C
:10083A00EE005E210430FB008E30FC001230FD0019
:10084A00FD0B252CFC0B252CFB0B252C0000E10AAB
:10085A00182C0230EE005E210130EE005E210130DC
:10086A00E3000130E4004230E5003B230130E300BD
:10087A000F30E4002130E5003B23D501DF01E00120
:10088A00273083168100833083128E00F5308F0063
:10089A000C100B11D601D701A8308B00101481015E
:1008AA000C18582C552C8B0110100030DD0001302B
:1008BA00DE000730E200D60DD70D561080305706FD
:1008CA00F00080305E067002031D6D2C5D08560232
:1008DA000318762CDE0CDD0CDE135E1BDE17E2033A
:1008EA00632C80305E06F00080307002031D7F2C7E
:1008FA0002305D0203188B2C0130DD000030DE006F
:10090A002830831681008312E201912C2030620480
:10091A00831681008312E20A8E0180308F000C1048
:10092A000B11D601D701A0308B00101481010C18CD
:10093A009F2C9C2C8B0110100108DB00DC0156084F
:10094A00E3005708E4000030E41BFF30E500E6004E
:10095A006508E6006408E5006308E400E3015B0853
:10096A00F0005C08F1000030F11BFF30F200F300E8
:10097A007008E30771080318710FE4077208031877
:10098A00720FE50773080318730FE6076208F00091
:10099A0070080319D72CE30DE40DE50DE60D63107D
:1009AA00FF3ECE2CA3225508031DE72C8030F00011
:1009BA00803060067002031DE42C5F08D03C031CE3
:1009CA00E72C022D8B010130EE005E210130E3009D
:1009DA000230E4002430E5003B230630FB001330EC
:1009EA00FC00AD30FD00FD0BF82CFC0BF82CFB0BCA
:0E09FA00F82C000000000612012D452C032DE4
:100A780021308400323083120313F0000930D30090
:080A88000530D4007B230800B7
:060A120048347A34003480
:100A180050346F3477346534723420344F3446346C
:0A0A280046342E342E342E340034F0
:100A32004634723465347134753465346E346334DB
:100A4200793443346F3475346E34743465347234AB
:020A520000346E
:060A540046343D3400347D
:100A5A0061347534643469346F342E3472346934D1
:0C0A6A006E3467342E346C347434003465
:02400E00182177
:00000001FF
